:020000040800F2
:1000000000060020E5010008090F00080D0F000898
:10001000650F00080D0F0008390F0008E701000800
:10002000E7010008E7010008E7010008D9290008F6
:10003000E7010008E7010008E7010008E701000800
:10004000E7010008E7010008E7010008E7010008F0
:10005000E7010008E70100088D3A0008B93A0008F6
:10006000E53A0008113B00083D3B0008E7010008A5
:10007000E7010008E7010008E7010008E7010008C0
:10008000E7010008E7010008E7010008E7010008B0
:10009000E7010008E7010008E7010008693B0008E4
:1000A000E7010008E7010008E7010008E701000890
:1000B00001390008E7010008E7010008E70100082E
:1000C000E7010008E7010008E7010008E701000870
:1000D000E701000835110008E70100084911000890
:1000E000D13B0008E7010008E7010008E70100082C
:1000F000E7010008E7010008E7010008E701000840
:10010000E7010008E7010008E7010008E70100082F
:100110005D11000871110008E7010008E7010008FF
:10012000E7010008E7010008E7010008E70100080F
:10013000E7010008E7010008E7010008E7010008FF
:10014000E7010008E7010008E70100081D31000889
:10015000E7010008E7010008E70100088511000831
:10016000E7010008E7010008E7010008E7010008CF
:10017000E7010008E7010008E7010008E7010008BF
:10018000E7010008E7010008E7010008E7010008AF
:10019000E7010008E7010008E7010008E70100089F
:1001A000E7010008E7010008E7010008E70100088F
:1001B000E7010008E7010008E7010008E70100087F
:1001C000E7010008E7010008E7010008E70100086F
:1001D000E7010008E7010008E7010008E70100085F
:1001E000D10E000802E000F000F8FEE772B63948D0
:1001F00080F30888384880F3098838484EF608515B
:10020000CEF20001086040F20000CCF200004EF691
:100210003471CEF200010860BFF34F8FBFF36F8FD0
:1002200040F20000C0F2F0004EF68851CEF200011C
:100230000860BFF34F8FBFF36F8F4FF00000E1EE08
:10024000100A4EF63C71CEF200010860062080F3E1
:100250001488BFF36F8F02F01DFC03F0ADFA4FF06E
:1002600055301F491B4A91423CBF41F8040BFAE745
:100270001C49194A91423CBF41F8040BFAE71A495C
:100280001A4A1B4B9A423EBF51F8040B42F8040B2A
:10029000F8E700201749184A91423CBF41F8040B87
:1002A000FAE702F0FBFB03F0E3FA144C144DAC4206
:1002B00003DA54F8041B8847F9E700F041F8114CC1
:1002C000114DAC4203DA54F8041B8847F9E702F0F9
:1002D000E3BB000000060020002200200000000810
:1002E00000000020000600204040000800220020FE
:1002F0002822002028220020EC390020E0010008FC
:10030000E4010008E4010008E40100082DE9F04FD1
:100310002DED108AC1F80CD0C3689D46BDEC108A43
:10032000BDE8F08F002383F311882846A047002002
:1003300001F07AFFFEE701F0FBFE00DFFEE70000C0
:100340001A4B7F2270B500241A700F225C709C70CB
:10035000DC701C715C719C71DC711C725C729A7235
:10036000DC7202F00BFB064602F030FB054650B98A
:100370000F4B9E4217D001339E4241F2883412BF88
:10038000054600240125002002F002FB0DB100F01B
:1003900059F800F03FFD00F0B5FB204600F0B0F842
:1003A00000F050F8F9E70446EDE700BF28220020EE
:1003B000010007B008B500F071FBA0F1200358421E
:1003C000584108BD07B5054B02211B88ADF8043024
:1003D00001A800F081FB03B05DF804FBB83C000805
:1003E00010B5202383F311881248C3680BB101F0C4
:1003F000B7FF0023104A0F484FF47A7101F05EFFF7
:10040000002383F311880D4C236813B12368013B4B
:100410002360636813B16368013B6360084B1B781A
:1004200033B9636823B9022000F05AFC32236360B9
:1004300010BD00BF34220020E1030008502300203B
:100440004822002010B5254B254953F8042F0132CE
:1004500000D110BD8B42F8D1224C234B22689A4226
:100460003AD9224B9B6803F1006303F580339A422B
:1004700032D2002000F060FB1D4B0220187000F00B
:1004800021FC1C4B1A6C00221A64196E1A66196E34
:10049000596C5A64596E5A665A6E5A6942F0800213
:1004A0005A615A6922F080025A615A691A6942F007
:1004B00000521A611A6922F000521A611B6972B661
:1004C0000D4A0E4B13601B682268202181F31188AE
:1004D0009D4683F30888104710BD00BFFCFF00084D
:1004E0001C00010804000108FFFF0008282200206A
:1004F000482200200038024008ED00E0000001081A
:100500002DE9F04F99B0B94D00902022FF2110A89D
:10051000AC6800F021FCB64A01951378A3B9B54840
:100520000121C3601170202383F31188C3680BB1CC
:1005300001F016FF0023B04AAE484FF47A7101F083
:10054000BDFE002383F31188009BAC4A03B1136006
:10055000AB4B009D029300261E705660B246374694
:10056000B146012000F0AEFB002D00F02582A34B28
:100570001B68002B40F0208219B0BDE8F08F0220EC
:10058000FFF718FF002840F01082009B002E08BFE4
:100590001D469C4B02211B88ADF82C300BA800F0A7
:1005A0009BFADEE74FF47A7000F078FAB0F10008B9
:1005B000EBDB0220FFF7FEFE0028E6D008F1FF3853
:1005C000B8F1040F00F2F381DFE808F0031E2124E4
:1005D000270018A8052340F8343D042100F07CFAD8
:1005E000012303FA08F848EA0A0A5FFA8AFA4FF088
:1005F000000900F005FC27B10AF00B030B2B08BF24
:100600000025FFF7DFFEACE704217848E6E7042188
:100610007D48E3E704217D48E0E74FF01C094846A8
:1006200000F08CFA09F104090B9004210BA800F0EA
:1006300053FAB9F12C0FF2D1D2E7002FA5D00AF06E
:100640000B030B2BA1D10220FFF7B4FE804600283C
:100650009BD001206A4E00F06FFA0220307000F04B
:1006600031FB00275FFA87FB584600F075FA054614
:1006700088B1584600F080FA01370028F2D146468A
:100680000025634B02211B88ADF82C300BA800F02D
:1006900023FA474665E701230220337000F004FB8C
:1006A0002C46019B9B689C4206D2204600F046FAED
:1006B0000130E4D10434F4E7029B00241C704F4B5A
:1006C00046465C604746254693E7002F3FF45DAF02
:1006D0000AF00B030B2B7FF458AF029B022018701B
:1006E00000F0F0FA322000F0D9F9B0F1000BFFF67B
:1006F0004CAF1BF003087FF448AF019B996804EBF3
:100700000B028A423FF641AFBBF5807F3FF63DAF1B
:10071000404A0392D8450FDA4FF47A7000F0BEF9E0
:10072000049004990029FFF630AF039A049908F861
:10073000021008F10108ECE7C820FFF73BFE8046F5
:1007400000283FF422AF1F2C11D8C4F120075F45C9
:1007500028BF5F4610AB24F003003A462D491844E9
:1007600000F0D0FA3A46FF212A4800F0F5FA4FEAA5
:10077000AB03DAB227490393204600F0F5FA0746A7
:1007800000283FF47EAF039B04EB830431E7022093
:10079000FFF710FE00283FF4F8AE00F013FA00282F
:1007A0003FF4F3AE4FF000084346019A926890453B
:1007B00032D2B8F11F0F12D8109A01320FD028F0A0
:1007C000030218A90A4452F8202C0B92184604225E
:1007D0000BA900F0DBFB08F104080346E5E74046FF
:1007E000039300F0ABF9039B0B90EFE72822002066
:1007F0004C23002034220020E10300085023002075
:1008000048220020BA3C00082C2200203022002080
:10081000BC3C00084C22002018A8042140F84C3DA4
:1008200000F05AF9E5E618A8002340F8343D6421A9
:1008300000F048F900287FF4A8AE0220FFF7BAFDC7
:1008400000283FF4A2AE0B9800F0A8F918AB43F8CB
:10085000480D04211846E3E718A8002340F8343D6A
:10086000642100F02FF900287FF48FAE0220FFF7FB
:10087000A1FD00283FF489AE0B9800F09DF918AB5C
:1008800043F8440DE5E70220FFF794FD00283FF40C
:100890007CAE00F0A7F918AB43F8400DD9E7022071
:1008A000FFF788FD00283FF470AE0BA9142000F07C
:1008B0009FF9804618A8042140F83C8D00F00CF9FF
:1008C00041460BA8ACE7322000F0E8F8B0F1000890
:1008D000FFF65BAE18F0030F7FF457AE019A9268F3
:1008E00008EB090393423FF650AE0220FFF762FD8A
:1008F00000283FF44AAE28F00308C844C1453FF43D
:1009000078AE484600F01AF904210A900AA800F0CF
:10091000E3F809F10409F1E74FF47A70FFF74AFDB3
:1009200000283FF432AE00F04DF9002842D0109B71
:1009300001330BD0082210A9002000F015FA00287E
:1009400038D02022FF2110A800F006FAFFF73AFD68
:10095000364801F06FFC0FE6002F3FF416AE0AF0A8
:100960000B030B2B7FF411AE18A8002340F8343D85
:10097000642100F0A7F8804600287FF406AE02202C
:10098000FFF718FD00283FF400AE0390FFF71AFDB3
:1009900041F2883001F04EFC0B9800F079FA00F03B
:1009A0002FFA039B45461F46DBE5074621E64FF03D
:1009B0000009EAE5B84664E6002000F06FF804900C
:1009C000049B002BFFF6D0AD012000F06DF9049BD5
:1009D000213B122B3FF6C5AD01A252F823F000BF18
:1009E0007F050008A50500083B0600086305000810
:1009F0006305000863050008CB060008C708000867
:100A00008F07000827080008590800088708000811
:100A1000630500089F08000863050008190900081D
:100A2000F30500086305000859090008A0860100C5
:100A30002DE9F84F4FF47A75DFF85880DFF85890B9
:100A400007460E465543002498F900305A1C5FFAB9
:100A500084FA01D0A34210D159F824000368324629
:100A6000D3F820B039462B46D847864205D1084BEB
:100A700083F800A00120BDE8F88F0134062CE3D1F3
:100A80004FF4FA7001F0D6FB0020BDE8F88F00BFEC
:100A90009823002000220020FC3C000807B502AB90
:100AA000002203F8012D012102461846FFF7C0FF7E
:100AB00020B19DF8070003B05DF804FB4FF0FF3054
:100AC000F9E700000A4608B50421FFF7B1FF80F0FE
:100AD0000100C0B2404208BD30B4074B1A78074B42
:100AE00053F822402368DD69054B0A46AC460146AF
:100AF000204630BC604700BF98230020FC3C000823
:100B0000A086010070B501F03DFE094C094E208021
:100B1000002530682388834208D901F02DFE336810
:100B200005440133B5F5803F3360F2D370BD00BF9B
:100B30009A2300205823002001F0D2BE00F100606B
:100B400000F580300068704700F10060920000F509
:100B5000803001F05DBE0000054B1A68054B1B8814
:100B60009B1A834202D9104401F006BE0020704750
:100B7000582300209A23002038B5074D04462868E2
:100B8000204401F001FE28B928682044BDE838401F
:100B900001F012BE38BD00BF5823002010F003033F
:100BA00008D1B0F5047F05D200F10050A0F508404F
:100BB0000068704700207047014BC058704700BF65
:100BC000107AFF1F064991F8243033B10023082220
:100BD000086A81F82430FFF7B7BF0120704700BFD3
:100BE0005C230020014B1868704700BF002004E020
:100BF00070B52A4B1C68C4F30B03240C63B140F29C
:100C00001342934231D040F2194293422FD040F226
:100C1000214293422DD10323214A0C2505FB0323B6
:100C20005D6893F9082042F201039C4224D0B4F598
:100C3000805F23D041F201039C4221D041F20303A3
:100C40009C421FD041F207039C4208BF3122441E40
:100C50000C44013D0B46A3421ED215F9016F581CEE
:100C600096B1034600F8016CF5E70123D4E70223AF
:100C7000D2E73F220B4DD6E73322E3E74122E1E7FB
:100C80005A22E4E75922E2E72C2584421D7001D95B
:100C9000981C5A70401A70BD1846FBE7002004E00B
:100CA000CC3C0008C03C0008022804D14FF0804230
:100CB000034B9A6170470128FCD14FF00052F7E7CF
:100CC00000000240022804D14FF48042034B9A6195
:100CD00070470128FCD14FF40052F7E700000240B2
:100CE000022805D1064A536983F480435361704753
:100CF0000128FCD1024A536983F40053F6E700BF90
:100D00000000024010B50023934203D0CC5CC454D1
:100D10000133F9E710BD000030B5441E14F9010F8E
:100D20000B4660B193F90050854201F1010106D1F3
:100D30001AB993F90020801A30BD013AEEE7002A73
:100D4000F7D1104630BD000002460346981A13F949
:100D5000011B0029FAD1704702440346934202D096
:100D600003F8011BFAE770472DE9F047234C94F88C
:100D7000243005468846174683BB2E46DFF87C9014
:100D8000C7B394F824302BB92022FF2148462662AD
:100D9000FFF7E2FF94F82400C0F10805BD4228BF28
:100DA0003D465FFA85FAAD0041462A4604EB8000D5
:100DB000FFF7A8FF94F82430A7EB0A079A445FFADC
:100DC0008AFABAF1080F2E44A844FFB284F824A08E
:100DD000D6D1FFF7F7FE0028D2D108E0266A06EB4D
:100DE0008306B042CAD0FFF7EDFE0028C5D100202F
:100DF000BDE8F0870120BDE8F08700BF5C2300203C
:100E0000024B1A78024B1A70704700BF98230020DB
:100E100000220020F8B5184C1848194D194E174FEC
:100E200000F01EFD2146154800F046FD24681648D6
:100E3000626DD2F8043843F00203C2F8043801F0BE
:100E4000F9F92046114900F043FE626DD2F80438EA
:100E500023F00203C2F804384FF4E1332B6000247E
:100E600056F82400B84202D0294600F057FC01345D
:100E7000062CF5D1F8BD00BF143E00081832002042
:100E800084230020FC3C000840420F003C3E000848
:100E900038B50B4B1A780B4B53F822400A4B9C4247
:100EA00005460CD0094B002118461422FFF754FFC9
:100EB000056001462046BDE8384000F02FBC38BD33
:100EC00098230020FC3C00081832002084230020D6
:100ED00070B50A4C1C26324600212046FFF73CFF25
:100EE0000125074B6360657032460021A019FFF7AA
:100EF00033FF044B25776577236270BD9C23002068
:100F00000E0002400D000240FEE7000000B59BB05D
:100F1000EFF3098168226846FFF7F4FEEFF30583DB
:100F2000044B9A6BDA6A9A6A9A6A9A6A9A6A9A6A15
:100F30009B6AFEE700ED00E000B59BB0EFF309818E
:100F400068226846FFF7DEFEEFF30583044B9A6BD9
:100F50009A6A9A6A9A6A9A6A9A6A9B6AFEE700BFD4
:100F600000ED00E000B59BB0EFF309816822684610
:100F7000FFF7C8FEEFF30583034B5A6B9A6A9A6A30
:100F80009A6A9A6A9B6AFEE700ED00E030B5084D68
:100F90000A4491420BD011F8013B09245840013C0E
:100FA000F7D040F300032B4083EA5000F7E730BD51
:100FB0002083B8ED002304491A465A50C818083354
:100FC000802B4260F9D17047D42300200268436827
:100FD0001143016003B1184770470000024AD3680B
:100FE00043F0C003D360704700100140024AD36849
:100FF00043F0C003D360704700480040024AD36802
:1010000043F0C003D3607047004C0040024AD368ED
:1010100043F0C003D360704700500040024AD368D9
:1010200043F0C003D3607047001401402DE9F04144
:10103000D0F85C62F7683368DA0505469CB20DD5D6
:10104000202383F311884FF400710430FFF7BEFFB3
:101050006FF480733360002383F31188202383F3BC
:10106000118805F1040814F02F0333D183F311889C
:10107000380615D5210613D5202383F3118805F1F1
:10108000380000F0A9FA002846DA0821281DFFF7E9
:101090009DFF4FF67F733B40F360002383F311887D
:1010A0007A060ED563060CD5202383F31188EA6CEB
:1010B0002B6D9A4202D12B6C002B2FD1002383F38E
:1010C0001188D5F86422D368002B31D01069BDE8AF
:1010D000F0411847230713D014F0080F0CBF00216C
:1010E0008021E00748BF41F02001A20748BF41F03E
:1010F0004001630748BF41F480714046FFF766FF37
:10110000A406736805D595F860122846194000F0CA
:1011100013FB3468A4B2A6E77060BEE727F040076F
:101120003F041021281D3F0CFFF750FFF760C5E773
:10113000BDE8F08108B50348FFF778FFBDE8084037
:1011400001F07EBC5424002008B50348FFF76EFF71
:10115000BDE8084001F074BCBC26002008B5034877
:10116000FFF764FFBDE8084001F06ABC24290020B5
:1011700008B50348FFF75AFFBDE8084001F060BC1E
:101180008C2B002008B50348FFF750FFBDE808404E
:1011900001F056BCF42D002010B5174C174A20461C
:1011A000002100F099FA164BC4F85C32154C164A2F
:1011B0002046002100F090FA144BC4F85C32144C25
:1011C000144A2046002100F087FA134BC4F85C3221
:1011D000124C134A2046002100F07EFA114BC4F84D
:1011E0005C32114C114A0021204600F075FA104B78
:1011F000C4F85C3210BD00BF54240020DD0F00088D
:1012000000100140BC260020ED0F000800480040FF
:1012100024290020FD0F0008004C00408C2B0020EA
:101220000D10000800500040F42D00201D10000893
:101230000014014038B5494D037C002918BF0D4604
:10124000012B0446C0F8645210D1454B984242D15C
:10125000444B5A6C42F010025A645A6E42F010022B
:101260005A665B6E0B21252000F08EF83E4BD4F8B9
:101270005C229A422B6802D03C498A426BD13C499D
:1012800001EB5301B1FBF3F3A988080442BF23F03B
:10129000070003F0070343EA40039360EB8843F041
:1012A00040039BB213612B8943F001039BB253614E
:1012B00041F4045343F02C03D36001F4A051002304
:1012C0001360B1F5806F136853680CBF7F23FF2351
:1012D00084F8603238BD274B98420CD1214B1A6CF0
:1012E00042F480221A641A6E42F480221A661B6E3F
:1012F0000B212720B8E7204B98420CD1194B1A6CD0
:1013000042F400221A641A6E42F400221A661B6E1E
:101310000B213420A8E7194B98420CD1114B1A6CC1
:1013200042F480121A641A6E42F480121A661B6E1E
:101330000B21352098E7124B984297D1094B5A6CF4
:1013400042F020025A645A6E42F020025A665B6EE6
:101350000B21472088E70B4992E700BF343D000886
:1013600054240020003802400010014000140140C5
:1013700000BD0105BC260020242900208C2B002064
:10138000F42D002080DE800200F1604300F01F0297
:10139000400903F5614309018000C9B200F16040D2
:1013A00083F8001300F5614001239340C0F88031B9
:1013B00003607047F8B5154682680669AA420B4675
:1013C000816938BF8568761AB542044607D2184647
:1013D0002A46FFF797FCA3692B44A3610DE011D9BE
:1013E00032461846FFF78EFCAF1B3A46E1683044A0
:1013F000FFF788FCE2683A44A261A3685B1BA36024
:101400002846F8BD18462A46FFF77CFCE368E4E767
:1014100083682DE9F041044693421546266938BF9A
:1014200085684069361AB5420F4606D22A46FFF74C
:1014300069FC63692B4463610DE012D93246A5EB68
:101440000608FFF75FFC4246B919E068FFF75AFC4F
:10145000E26842446261A3685B1BA3602846BDE862
:10146000F0812A46FFF74EFCE368E4E710B50A4432
:101470000024C361029B006040608460C1608161A0
:1014800041610261036210BD08B5826943699342FC
:1014900001D1826882B98268013282605A1C42613D
:1014A0001970426903699A4201D3C36843610021FC
:1014B00000F0DCFE002008BD4FF0FF3008BD00004A
:1014C00070B5202304460E4683F31188A568A5B1A4
:1014D000A368A269013BA360531CA361157822692C
:1014E000934224BFE368A361E3690BB120469847A8
:1014F000002383F31188284670BD3146204600F052
:10150000A5FE0028E2DA85F3118870BD2DE9F74FBA
:1015100005460F4690469A46D0F81C90202686F342
:1015200011884FF0000B144664B122463946284614
:10153000FFF740FF034668B95146284600F086FE93
:101540000028F1D0002383F31188A8EB040003B036
:10155000BDE8F08FB9F1000F03D001902846C847CD
:10156000019B8BF31188E41A1F4486F31188DBE793
:10157000C16081614161C3611144009B00604060B2
:101580008260016103627047F8B504460E46174653
:10159000202383F31188A568A5B1A368013BA3604C
:1015A00063695A1C62611E70236962699A4224BF92
:1015B000E3686361E3690BB120469847002080F33C
:1015C0001188F8BD3946204600F040FE0028E2DAD6
:1015D00085F31188F8BD0000836942699A4210B50D
:1015E00001D182687AB98268013282605A1C8261B4
:1015F0001C7803699A4201D3C3688361002100F01B
:1016000035FE204610BD4FF0FF3010BD2DE9F74FDD
:1016100005460F4690469A46D0F81C90202686F341
:1016200011884FF0000B144664B122463946284613
:10163000FFF7EEFE034668B95146284600F006FE65
:101640000028F1D0002383F31188A8EB040003B035
:10165000BDE8F08FB9F1000F03D001902846C847CC
:10166000019B8BF31188E41A1F4486F31188DBE792
:10167000026843681143016003B1184770470000D6
:101680001430FFF743BF00004FF0FF331430FFF773
:101690003DBF00003830FFF7B9BF00004FF0FF3307
:1016A0003830FFF7B3BF00001430FFF709BF000068
:1016B0004FF0FF311430FFF703BF00003830FFF761
:1016C00063BF00004FF0FF323830FFF75DBF00000E
:1016D00000207047FFF760BD37B50F4B0360002354
:1016E00043608360C3600123044603741546009081
:1016F0000B464FF4807200F15C011430FFF7B6FE28
:1017000000942B464FF4807204F5AE7104F138005A
:10171000FFF72EFF03B030BD483D000810B5202371
:10172000044683F31188FFF785FD02232374002309
:1017300083F3118810BD000038B5C36904460D4617
:101740001BB904210844FFF793FF294604F1140054
:10175000FFF79AFE002806DA201D4FF48061BDE8ED
:101760003840FFF785BF38BD026843681143016008
:1017700003B118477047000013B5446BD4F8943494
:101780001A681178042915D1217C022912D11979FE
:10179000128901238B4013420CD101A904F14C00A2
:1017A00001F00EFFD4F89444019B21790246206891
:1017B00000F0DAF902B010BD143001F091BE000063
:1017C0004FF0FF33143001F08BBE00004C3001F0BD
:1017D00063BF00004FF0FF334C3001F05DBF0000ED
:1017E000143001F05FBE00004FF0FF31143001F003
:1017F00059BE00004C3001F02FBF00004FF0FF3207
:101800004C3001F029BF0000D0F8942438B513689B
:1018100019780429054601D0012038BD017C022930
:10182000FAD112795C89012090400440F4D105F18D
:10183000140001F0F1FD02460028EDD0D5F89454D3
:101840004FF480732868697900F07CF9204638BD30
:10185000406BFFF7D9BF00000020704770470000C1
:101860007FB5124B0360002343608360C360012592
:1018700002260F4B057404460290019300F1840286
:10188000294600964FF48073143001F0A1FD094BF6
:101890000193029400964FF4807304F52372294655
:1018A00004F14C0001F068FE04B070BD703D00080A
:1018B00051180008791700080B68202282F311885C
:1018C0000A7903EB820290614A79093243F82200D7
:1018D0008A7912B103EB8203986102230374C0F882
:1018E0009414002383F311887047000038B5037FF8
:1018F000044613B190F85430ABB9201D01250221E4
:10190000FFF732FF04F1140025776FF0010100F0BA
:10191000B9FC84F8545004F14C006FF00101BDE8AB
:10192000384000F0AFBC38BD10B50121044604308A
:10193000FFF71AFF0023237784F8543010BD00000E
:1019400038B504460025143001F05AFD04F14C006E
:10195000257701F029FE201D84F854500121FFF75E
:1019600003FF2046BDE83840FFF74EBF90F84430F3
:1019700003F06003202B19D190F84520212A0AD0CA
:10198000222A4FF000030ED0202A0FD1084A82638A
:101990000722C26304E0064B83630723C36300236B
:1019A0000364012070478363C363F9E70020704735
:1019B00001220020D0F8943437B51A681178042930
:1019C00004461AD1017C022917D119791289012301
:1019D0008B40134211D100F14C05284601F0A4FEC2
:1019E00058B101A9284601F0EBFDD4F89444019BBD
:1019F00021790246206800F0B7F803B030BD00003E
:101A000000EB8103F7B59C6905460E46F4B120232F
:101A100083F3118805EB8607201D0821FFF7A4FE3C
:101A2000FB685B691B684C3413B1204601F0D6FD9E
:101A300001A9204601F0C4FD024648B1019B314690
:101A4000284600F091F8002383F3118803B0F0BD1D
:101A5000FB685A691268002AF5D01B8A013B1340C3
:101A6000F1D105F14402EAE7093138B550F82140D7
:101A7000DCB1202383F31188D4F8942413685279BD
:101A800003EB8203DB689B695D6845B10421601844
:101A9000FFF76AFE294604F1140001F0C7FC204656
:101AA000FFF7B2FE002383F3118838BD70470000B2
:101AB00001F086B80123037000234360C361836291
:101AC0000362C36243620363038143817047000082
:101AD00038B50446202383F3118800254160C56092
:101AE00005614561856101F07BF80223237085F370
:101AF000118838BD70B500EB810305465069DA6086
:101B00000E46144618B110220021FFF725F9A069EE
:101B100018B110220021FFF71FF931462846BDE811
:101B2000704001F027B90000028902F00102028131
:101B3000428902F001024281002202614261826117
:101B400001F0ACB9F0B400EB81044789E4680125E9
:101B5000A4698D403D43458123600023A2606360FA
:101B6000F0BC01F0C7B90000F0B400EB81040789B4
:101B7000E468012564698D403D43058123600023AD
:101B8000A2606360F0BC01F041BA000070B50223AE
:101B9000002504460370A0F84C5080F84E5080F8A1
:101BA0004F5005814581C56005614561856180F8BB
:101BB000345001F07BF863681B6823B12946204646
:101BC000BDE87040184770BD037880F85030052399
:101BD000037043681B6810B504460BB10421984795
:101BE00000232381638110BD436890F850201B6857
:101BF00002700BB1052118477047000090F834308F
:101C000070B5044613B1002380F8343004F1440267
:101C1000204601F065F963689B6863BB94F8445003
:101C200015F0600615D194F8453005F07F0545EABA
:101C3000032540F202339D4200F00E815BD8022D55
:101C400000F0DC803FD8002D00F08780012D00F0EF
:101C5000CF800021204601F09DFB0021204601F0AD
:101C60008FFB63681B6813B1062120469847062343
:101C700084F8343070BD204698470028CED094F8C0
:101C80004B2094F84A3043EA0223E26B934238BF78
:101C9000E36394F94430E56B002B4FF0200380F2AE
:101CA000FD80002D00F0EC80092284F8342083F3BD
:101CB00011880021E36BA26B2046FFF755FF00233C
:101CC00083F3118870BDB5F5817F00F0B180B5F563
:101CD000407F49D0B5F5807FBBD194F84630012BC9
:101CE000B7D1B4F84C3023F00203A4F84C30A6630B
:101CF000E6632664C3E740F201639D421ED8B5F552
:101D0000C06F3BD2B5F5A06FA3D1B4F84430B3F5A2
:101D1000A06F0ED194F8463084F84E30204601F082
:101D20001DF863681B6813B10121204698470323FF
:101D300023700023A363E3632364A0E7B5F5106F6A
:101D400032D040F602439D4252D0B5F5006F80D1AB
:101D500004F14F03A363012324E004F14C03A363C4
:101D60000223E36325648AE794F84630012B7FF46D
:101D700070AFB4F84C3043F00203B6E794F8492052
:101D8000616894F848304D6894F8471043EA02239C
:101D9000204694F84620A84700283FF45AAF4368ED
:101DA000A3630368E363A4E72378042B10D1202303
:101DB00083F311882046FFF7B7FE86F31188636826
:101DC00084F84F601B68032121700BB120469847AF
:101DD00094F84630002BACD084F84F3004232370A5
:101DE00063681B68002BA4D0022120469847A0E717
:101DF000374BA3630223E36300239DE794F8481065
:101E000011F0800F204601F00F010ED001F05AF8BA
:101E1000012806D002287FF41CAF2E4BA363E06399
:101E200067E72D4BA363E56363E701F03DF8EFE758
:101E300094F84630002B7FF40CAF94F8483013F040
:101E40000F013FF476AF1A06204602D501F0B6FA2C
:101E50006FE701F0A9FA6CE794F84630002B7FF4A5
:101E6000F8AE94F8483013F00F013FF462AF1B0650
:101E7000204602D501F08EFA5BE701F081FA58E7BF
:101E8000142284F8342083F311882B462A462946ED
:101E90002046FFF757FE85F3118870BD5DB115220E
:101EA00084F8342083F311880021E36BA26B204671
:101EB000FFF748FE03E70B2284F8342083F31188F0
:101EC0002B462A4629462046FFF74EFEE3E700BF91
:101ED000A03D0008983D00089C3D000838B590F8EA
:101EE00034300446152B29D8DFE803F03E28282893
:101EF00028283E28280B2939282828282828282857
:101F00003E3E90F84B1090F84A20C36B42EA012203
:101F10009A4214D9C268128AB3FBF2F502FB153556
:101F20006DB9202383F311882B462A462946FFF7F3
:101F30001BFE85F311880A2384F8343038BD14233E
:101F400084F83430202383F3118800231A4619467D
:101F50002046FFF7F7FD002383F3118838BD036C9B
:101F600003B198470023E7E7002101F013FA0021AD
:101F7000204601F005FA63681B6813B1062120466C
:101F800098470623D8E7000090F83420152A38B582
:101F9000044622D80123934040F6416213421DD1EA
:101FA00013F480150FD19B0217D50B2380F8343022
:101FB000202383F311882B462A462946FFF7D4FDB8
:101FC00085F3118838BDC3689B695B682BB9036CC6
:101FD00003B19847002384F8343038BD002101F064
:101FE000D9F90021204601F0CBF963681B6813B1D1
:101FF0000621204698470623EDE70000024B002209
:102000001B605B609A6070475C30002000230374A3
:102010008268054B1B6899689142FBD25A6803603D
:1020200042601060586070475C30002008B5202383
:1020300083F31188037C032B05D0042B0DD02BB91F
:1020400083F3118808BD436900221A604FF0FF3303
:102050004361FFF7DBFF0023F2E790E80C001A6012
:1020600002685360F2E70000002303748268054BA6
:102070001B6899689142FBD85A68036042601060FF
:10208000586070475C300020054B19690874186867
:1020900002681A605360186101230374FEF736B9B1
:1020A0005C30002030B54B1C87B005460A4C10D080
:1020B00023690A4A01A800F001F92846FFF7E4FF66
:1020C000049B13B101A800F04BF92369586907B0CC
:1020D00030BDFFF7D9FFF8E75C3000202D20000865
:1020E00038B50C4D41612B6981689A68914204466C
:1020F00003D8BDE83840FFF789BF1846FFF7B4FFA3
:1021000001232C61014623742046BDE83840FEF7C8
:10211000FDB800BF5C300020044B1A681B69906852
:102120009B68984294BF0020012070475C300020DB
:1021300010B5084C236820691A6822605460012297
:1021400023611A74FFF790FF01462069BDE8104033
:10215000FEF7DCB85C300020FEE7000010B50C4C48
:10216000FFF74CFF00F09CF880220A49204600F05F
:1021700021F8012344F8180C037400F03DFC0023FF
:1021800083F3118862B60448BDE8104000F034B80B
:1021900084300020A43D0008AC3D000800F01AB9CE
:1021A000034B59685A68521A9042FBD8704700BFD7
:1021B000001000E082600222027400224274704724
:1021C0008368A3F17C0243F80C2C026943F83C2C91
:1021D000426943F8382C074A43F81C2CC26843F87C
:1021E000102C022203F8082C002203F8072CA3F17C
:1021F000180070472503000810B5202383F31188C9
:10220000FFF7DEFF00210446FFF76AFF002383F398
:102210001188204610BD0000024B1B6958610F2039
:10222000FFF732BF5C300020202383F31188FFF7D3
:10223000F3BF000008B50146202383F3118808206E
:10224000FFF730FF002383F3118808BD49B1064B27
:1022500042681B6918605A60136043600420FFF7EE
:1022600021BF4FF0FF3070475C3000200368984278
:1022700006D01A680260506059611846FFF7C6BE62
:102280007047000038B504460D462068844200D1EE
:1022900038BD036823605C604561FFF7B7FEF4E773
:1022A000054B03F114025A619A614FF0FF32DA6173
:1022B00000221A62704700BF5C300020F8B5274F3B
:1022C0000361C2600D46044601F062FA3B46022DEE
:1022D00053F8142F294638BF02219A423E461D4624
:1022E0000AD138627C61BC61084422606260A160EE
:1022F000BDE8F84001F03ABAD7F820E0A0EB0E03B1
:102300005F181FD300279068834217D8376AAA4204
:102310001F44376201D0C01A906073699A68914275
:1023200019D85A682360626014605C60A160986884
:10233000411A99604FF0FF33F361F8BD97601B1AA3
:102340001268E0E793689F4203D20EEB070001F0AA
:102350001BFA3946E1E7891A1B68DFE75C30002089
:1023600038B51B4B01685A6990421D4603F11402AF
:102370000CD0446821600368002193425C60C16016
:1023800025D09A6881680A449A6038BD59614A60CC
:102390005B6900219342C16003D1BDE8384001F080
:1023A000EDB99A6881680A449A602C6A01F0F0F9E4
:1023B0006A699268001B824209D9111A012998BFE3
:1023C000821C286ABDE83840104401F0DDB938BDF0
:1023D0005C3000202DE9F84F204C0027656904F19E
:1023E0001406B84601F0D4F9236AA0EB030AAB68DF
:1023F00053451DD84FF02009236AAA68D5F80CB0C0
:1024000013442362AB68AAEB030A2B68B3425E60F5
:102410006361EF6001D101F0B1F988F31188286997
:10242000D84789F311886569AB689A45E4D2D9E742
:102430006369B34210D020629A68A2EB0A029A60E4
:10244000226AAB68821A9B1A022B2CBFC01802307A
:10245000BDE8F84F01F098B9BDE8F88F5C30002076
:1024600000207047FEE70000704700004FF0FF308B
:1024700070470000022906D0032906D0012906482A
:1024800018BF0020704705487047032A9ABF0448C8
:1024900000EBC20000207047983E00084C3E000848
:1024A0000822002070B59AB001AD064608462946BC
:1024B000144600F095F82846FEF746FCC0B2431CCF
:1024C0005B0086E818002370032363700023023446
:1024D0001946DAB2904204F1020401D81AB070BD74
:1024E000EA5C04F8022C04F8011C0133F1E7000057
:1024F00008B5202383F311880348FFF75BFA002314
:1025000083F3118808BD00BF1832002010B50446BF
:10251000052916D8DFE801F016150316161D20232D
:1025200083F311880E4A0121FFF7E4FA20460D4A91
:102530000221FFF7DFFA0C48FFF702FA002383F3CA
:10254000118810BD202383F311880748FFF7CEF9C7
:10255000F4E7202383F311880348FFF7E5F9EDE75B
:10256000CC3D0008F03D00081832002038B50C4D75
:102570000C4C0D492A4604F10800FFF793FF05F1C2
:10258000CA0204F110000949FFF78CFF05F5CA7271
:1025900004F118000649BDE83840FFF783BF00BFCB
:1025A000E0360020082200201C3E0008263E0008DD
:1025B000313E000870B5044608460D46FEF7C4FBE0
:1025C000C6B22046013403780BB9184670BD3246B6
:1025D0002946FEF7A1FB0028F3D1012070BD0000C1
:1025E0002DE9F04704460D46FEF7AEFB2C49C6B276
:1025F0002046FFF7DFFF08B10736F6B2294920462B
:10260000FFF7D8FF08B11036F6B2632E0BD8DFF80B
:102610009080DFF89090244FDFF898A0267846B994
:102620002E70BDE8F08721462846BDE8F04701F04E
:102630003BBB252E2FD1072241462046FEF76CFBDF
:1026400070B91A4B2A4603F10C0153F8040B42F8F7
:10265000040B8B42F9D11B88138007340E35DDE75C
:10266000082249462046FEF757FBA0B9104BAA1C8A
:1026700013F8011F09095345C95D02F8021C1978B6
:1026800001F00F0102F10202C95D02F8031CEFD153
:1026900018350834C2E72E7001340135BEE700BF9B
:1026A000B83E0008313E0008CF3E0008C03E00089A
:1026B0000F7AFF1F1B7AFF1FBFF34F8F024AD368A9
:1026C000DB03FCD4704700BF003C024008B5094B57
:1026D0001B7873B9FFF7F0FF074B1A69002ABFBFD9
:1026E000064A5A6002F188325A601A6822F48062FF
:1026F0001A6008BD3E390020003C024023016745B6
:1027000008B50B4B1B7893B9FFF7D6FF094B1A6935
:1027100042F000421A611A6842F480521A601A6844
:1027200022F480521A601A6842F480621A6008BD6E
:102730003E390020003C02400B2870B513D80B4AEC
:102740000B4C137863B90B4E4FF0006144F8231023
:1027500056F8235001330C2B2944F7D10123137071
:1027600054F8200070BD002070BD00BF70390020FB
:1027700040390020E03E0008014B53F8200070472C
:10278000E03E00080C2070470B2810B5044601D924
:10279000002010BDFFF7D0FF064B53F8243018443B
:1027A000C21A0BB9012010BD12680132F0D1043BEE
:1027B000F6E700BFE03E00080B2810B5044621D81C
:1027C000FFF77AFFFFF782FF0F4AF323D360C300BE
:1027D000DBB243F4007343F002031361136943F463
:1027E00080331361FFF768FFFFF7A6FF074B53F82D
:1027F000241000F0DDF8FFF783FF2046BDE810400D
:10280000FFF7C2BF002010BD003C0240E03E0008C0
:102810002DE9F84312F00103154640D18218B2F1B8
:10282000016F3CD22C4B1B6813F0010337D02B4CAB
:10283000FFF74CFFF323E360FFF73EFF40F2012771
:10284000032D01D9830713D0244C0F46401A40F2C0
:102850000118EB1B0B44012B00EB0706236924D85E
:1028600023F001032361FFF74BFF0120BDE8F8834C
:10287000236923F44073236123693B43236151F8A7
:10288000046B0660BFF34F8FFFF716FF03689E428D
:1028900008D0236923F001032361FFF731FF0020F3
:1028A000BDE8F883043D0430CAE723F44073236194
:1028B000236943EA08032361B94637F8023B3380B2
:1028C000BFF34F8FFFF7F8FE3688B9F80030B6B285
:1028D000B342BED0DDE700BF00380240003C0240FA
:1028E000084908B50B7828B153B9FFF7EFFE01236B
:1028F0000B7008BD23B1BDE808400870FFF700BFAA
:1029000008BD00BF3E39002010B50244064B043913
:10291000D2B2904200D110BD441C00B253F8200046
:1029200041F8040FE0B2F4E750280040104B30B5F6
:102930001C6F240407D41C6F44F400741C671C6FC4
:1029400044F400441C670B4C236843F480732360F9
:102950000244094B0439D2B2904200D130BD441C2C
:1029600000B251F8045F43F82050E0B2F4E700BF32
:1029700000380240007000405028004007B5012296
:1029800001A90020FFF7C0FF019803B05DF804FB28
:1029900013B50446FFF7F2FFA04206D002A90122B8
:1029A00041F8044D0020FFF7C1FF02B010BD000048
:1029B00070470000034B1B689B0042BF024B012283
:1029C0001A7070477438024071390020014B187832
:1029D000704700BF71390020EFF3098305494A6849
:1029E00022F001024A60683383F30988002383F3ED
:1029F0001188704730EF00E0202080F3118862B624
:102A00000B4B0C4AD96821F4E0610904090C0A4314
:102A10000949DA60CA6842F08072CA6007490A68E8
:102A200042F001020A601022DA7783F82200704730
:102A300000ED00E00003FA05F0ED00E0001000E01A
:102A400010B5202383F311880E4B5B6813F40063E9
:102A500014D0F1EE103AEFF30984683C4FF0807324
:102A6000E361094BDB68236684F30988FFF754FBB5
:102A700010B1064BA36110BD054BFBE783F3118832
:102A800010BD00BF00ED00E030EF00E037030008AC
:102A90003A03000870470000FEE70000084A094BAF
:102AA00009498B4204D3094A0021934205D3704758
:102AB00052F8040F43F8040BF3E743F8041BF4E760
:102AC00064400008EC390020EC390020EC3900208B
:102AD000836D70B5446D9E6800214FF0FF354A014B
:102AE000A3180131D3F800090028BEBFD3F80009AC
:102AF00040F08040C3F80009D3F8000B0028BEBFA7
:102B0000D3F8000B40F08040C3F8000BA3188E42AE
:102B1000C3F80859C3F8085BE1D24FF00113C4F8B9
:102B20001C3870BD890141F02001016103699B06D9
:102B3000FCD41220FFF734BB204B03EB80022DE9BD
:102B4000F047D2F80CE05D6DDEF81420461CD2F898
:102B500000C005EB063605EB4018516861450BD304
:102B6000D5F83428012303FA00F022EA0000C5F862
:102B700034081846BDE8F087BEF81040ACEB0103FE
:102B8000A34228BF2346D8F81849A4B2B3EB840F58
:102B900010D894681F46A4F1040959F804AFC6F888
:102BA00000A0042F01D9043FF7E71C440B449460B4
:102BB0005360D2E70020BDE8F08700BF74390020E1
:102BC00010B5054C2046FEF775FF4FF0A043636536
:102BD000024BA36510BD00BF74390020343F0008CC
:102BE0000378012B70B5054650D12A4B446D9842AD
:102BF0001BD1294B5A6B42F080025A635A6D42F046
:102C000080025A655A6D5A6942F080025A615A69C7
:102C100022F080025A610E2143205B69FEF7B4FB6B
:102C20001E4BE3601E4BC4F800380023C4F8003E7E
:102C3000C02323606E6D4FF40413A3633369002B2C
:102C4000FCDA012333610C20FFF7AAFA3369DB07B2
:102C5000FCD41220FFF7A4FA3369002BFCDA00261B
:102C6000A6602846FFF734FF6B68C4F81068DB687D
:102C7000C4F81468C4F81C684BB90A4BA3614FF040
:102C8000FF336361A36843F00103A36070BD064B8B
:102C9000F4E700BF743900200038024040140040BF
:102CA00003002002003C30C0083C30C0F8B5446D41
:102CB000054600212046FFF735FFA96D00234FF0A0
:102CC00001128F68C4F834384FF00066C4F81C282D
:102CD0004FF0FF3004EB431201339F42C2F800690A
:102CE000C2F8006BC2F80809C2F8080BF2D20B68F0
:102CF0006A6DEB65636210231361166916F01006A6
:102D0000FBD11220FFF74CFAD4F8003823F4FE630D
:102D1000C4F80038A36943F4402343F01003A361CF
:102D20000923C4F81038C4F814380A4BEB604FF08C
:102D3000C043C4F8103B084BC4F8003BC4F810690A
:102D4000C4F80039EB6D03F1100243F48013EA6517
:102D5000A362F8BD103F000840800010426D90F85B
:102D60004E10D2F8003823F4FE6343EA0113C2F890
:102D7000003870472DE9F0410EB200EB86080D4691
:102D8000D8F80C100F6807F00303022B50D0032B68
:102D900050D03D4A3D4F012B18BF1746446D4FEAB6
:102DA000451E04EB0E030022C3F8102B8A6905F1BF
:102DB000100C002A40D04A8A05F158035B013A43BF
:102DC000E2500123D4F81C2803FA0CF31343A64461
:102DD0004A69C4F81C380023CEF8103905F13F03C6
:102DE000002A39D00A8A898B9208012988BF4A4370
:102DF000C16D04EB8303561841EA0242C6652946B9
:102E00005A602046FFF78EFED8F80C301B8A43EA42
:102E100085531F4305F148035B01E7500123D4F8B4
:102E20001C2803FA05F51543C4F81C58BDE8F081C9
:102E3000174FB3E7174FB1E704EB4613D3F8002B56
:102E400022F40042C3F8002BD4F81C28012303FA13
:102E50000CF322EA0303BAE704EB83030E4A5A6039
:102E600004EB461629462046FFF75CFED6F80039EB
:102E700023F40043C6F80039D4F81C38012202FAC2
:102E800005F523EA0505CFE7008000100080041057
:102E90000080081000800C1000040002826D12688F
:102EA000C265FFF715BE00005831436D49015B58FC
:102EB00013F4004004D013F4001F14BF01200220BB
:102EC000704700004831436D49015B5813F40040DE
:102ED00004D013F4001F14BF01200220704700002B
:102EE00000EB8101CB68196A0B6813604B68536073
:102EF0007047000000EB810330B5DD68AA691368F4
:102F0000D36019B9402B84BF402313606B8A1468C7
:102F1000426D1C44013CB4FBF3F46343033323F0E0
:102F2000030302EB411043EAC44343F0C043C0F83B
:102F3000103B2B6803F00303012B09B20ED1D2F82A
:102F4000083802EB411013F4807FD0F8003B14BF27
:102F500043F0805343F00053C0F8003B02EB4112B2
:102F6000D2F8003B43F00443C2F8003B30BD000000
:102F70002DE9F041244D6E6D06EB40130446D3F865
:102F8000087BC3F8087B38070AD5D6F81438190728
:102F900006D505EB84032146DB6828465B68984725
:102FA000FA072FD5D6F81438DB072BD505EB8403A9
:102FB000D968CCB98B69488A5E68B6FBF0F200FB31
:102FC00012628AB91868DA6890420DD2121A83E840
:102FD0001400202383F311880B482146FFF78AFF52
:102FE00084F31188BDE8F081012303FA04F26B89B0
:102FF00023EA02036B81CB6823B121460248BDE876
:10300000F0411847BDE8F0817439002000EB8103DE
:1030100070B5DD68436D6C692668E6604A0156BB91
:103020001A444FF40020C2F810092A6802F0030283
:10303000012A0AB20ED1D3F8080803EB421410F4A7
:10304000807FD4F8000914BF40F0805040F0005059
:10305000C4F8000903EB4212D2F8000940F0044022
:10306000C2F80009D3F83408012202FA01F1014341
:10307000C3F8341870BD19B9402E84BF40202060B9
:1030800020682E8A841940F00050013C1A44B4FB99
:10309000F6F440EAC440C6E7F8B504461E48456D5C
:1030A00005EB4413D3F80869C3F80869F10717D58D
:1030B000D5F81038DA0713D500EB8403D9684B69CB
:1030C0001F68DA68974218D2D21B00271A605F6027
:1030D000202383F311882146FFF798FF87F3118897
:1030E000330617D5D5F834280123A340134211D055
:1030F0002046BDE8F840FFF71FBD012303FA04F2A4
:10310000038923EA020303818B68002BE8D0214660
:103110009847E5E7F8BD00BF7439002097482DE9CE
:10312000F84F456D6E69AB691E4016F4805F6E61A5
:10313000044605D0FEF72AFDBDE8F84FFFF780BC36
:10314000002E12DAD5F8003E8C489B071EBFD5F83A
:10315000003E23F00303C5F8003ED5F8043823F001
:103160000103C5F80438FEF73FFD370505D5834850
:10317000FFF7AEFC8148FEF727FDB0040CD5D5F86B
:10318000083813F0060FEB6823F470530CBF43F4B8
:10319000105343F4A053EB60310704D56368DB6838
:1031A0000BB176489847F2025AD4B3020CD5D4F842
:1031B0005480DFF8C8A100274FF00109A36D9B6878
:1031C000F9B28B4280F08780F70619D5616D0A6AE3
:1031D000C2F30A1702F00F0302F4F012B2F5802FC7
:1031E00000F0A180B2F5402F0AD104EB830301F572
:1031F0008051DB68186A00231A469F4240F087809E
:103200003003D5F8184813D5E10302D50020FFF7A5
:10321000AFFEA20302D50120FFF7AAFE630302D589
:103220000220FFF7A5FE270302D50320FFF7A0FE2B
:10323000750381D5E00702D50020FFF72DFFA10718
:1032400002D50120FFF728FF620702D50220FFF711
:1032500023FF23077FF570AF0320FFF71DFF6BE708
:10326000D4F85480DFF814A100274FF00109A36DB2
:103270009B685FFA87FB5B4597D308EB4B13D3F84A
:10328000002902F44022B2F5802F22D1D3F8002980
:10329000002A1EDAD3F8002942F09042C3F8002930
:1032A000D3F80029002AFBDB5946606DFFF73AFC92
:1032B000228909FA0BF322EA0303238104EB8B032F
:1032C000DB689B6813B15946504698475846FFF74C
:1032D00033FC0137CBE708EB4112D2F8003B03F493
:1032E0004023B3F5802F10D1D2F8003B002B0CDA2D
:1032F000628909FA01F322EA0303638104EB810383
:10330000DB68DB680BB150469847013756E79C07EE
:1033100008BF0A68072B98BF027003F101039CBF26
:10332000120A013069E7023304EB830201F5805190
:10333000526890690268D0F808C04068A2EB000E9D
:103340000022104697420AD104EB830463689B690C
:103350009A683A449A605A6817445F6050E712F0DE
:10336000030F08BF0868964588BF8CF8000002F17B
:10337000010284BF000A0CF1010CE3E7743900205C
:10338000436D03EB4111D1F8003B43F40013C1F846
:10339000003B7047436D03EB4111D1F8003943F412
:1033A0000013C1F800397047436D03EB4111D1F8A8
:1033B000003B23F40013C1F8003B7047436D03EB5F
:1033C0004111D1F8003923F40013C1F800397047D6
:1033D00030B5039C0172043304FB0325C361049BD5
:1033E00003630021059B00604060C160426102618F
:1033F0008561046242628162C162436330BD000044
:103400000022416A41610161C2608262C2626FF062
:103410000101FEF737BF000003694269934203D1FF
:10342000C2680AB100207047181D7047036919600F
:10343000C2680132C260C269134482690361934267
:1034400024BF436A03610021FEF710BF38B504466C
:103450000D46E3683BB16269131D1268A362134411
:10346000E362002038BD237A33B929462046FEF7AF
:10347000EDFE0028EDDA38BD6FF00100FBE700003B
:10348000C368C269013BC3604369134482694361F5
:10349000934224BF436A436100238362036B03B1F9
:1034A0001847704770B52023044683F31188866A55
:1034B0003EB9FFF7CBFF054618B186F311882846C1
:1034C00070BDA36AE26A13F8015BA362934202D360
:1034D0002046FFF7D5FF002383F31188EFE70000B4
:1034E0002DE9F84F04460E4690469946202787F36B
:1034F00011880025AA46D4F828B0BBF1000F09D1E5
:1035000049462046FFF7A2FF20B18BF311882846D9
:10351000BDE8F88FA16AE36AA8EB050B5B1A9B452F
:1035200028BF9B46BBF1400F1BD9334601F1400237
:1035300051F8040B43F8040B9142F9D1A36A4033CC
:103540004036A3624035A26AE36A9A4202D320461B
:10355000FFF796FF8AF311884545D8D287F3118883
:10356000C9E730465A46FDF7CDFBA36A5B445E448B
:10357000A3625D44E7E7000010B5029C01720433CA
:1035800003FB0421C36100238362C362039B0363C3
:10359000049B00604060C46042610261816104621A
:1035A0004262436310BD0000026AC260426A426127
:1035B000026100228262C2626FF00101FEF762BE08
:1035C000436902699A4203D1C2680AB10020704778
:1035D000184650F8043B0B6070470000C368C2698E
:1035E0000133C3604369134482694361934224BF3A
:1035F000436A43610021FEF739BE000038B5044636
:103600000D46E3683BB123691A1DA262E2691344C7
:10361000E362002038BD237A33B929462046FEF7FD
:1036200015FE0028EDDA38BD6FF00100FBE7000061
:1036300003691960C268013AC260C26913448269B1
:103640000361934224BF436A036100238362036BD7
:1036500003B118477047000070B5202304460E469A
:1036600083F31188856A35B91146FFF7C7FF10B19A
:1036700085F3118870BDA36A1E70A36AE26A0133E4
:103680009342A36204D3E16920460439FFF7D0FFD7
:10369000002080F3118870BD2DE9F84F04460D46D7
:1036A00091469A464FF0200888F311880026B346C9
:1036B000A76A4FB951462046FFF7A0FF20B187F314
:1036C00011883046BDE8F88FA06AE76AA9EB0603C7
:1036D0003F1A9F4228BF1F46402F1BD905F14003C8
:1036E00055F8042B40F8042B9D42F9D1A36A4033CE
:1036F000A3624036A26AE36A9A4204D3E169204693
:103700000439FFF795FF8BF311884E45D9D288F322
:103710001188CDE729463A46FDF7F4FAA36A3B44FF
:103720003D44A3623E44E5E7026943699A4203D1FE
:10373000C3681BB9184670470023FBE7836A002B58
:10374000F8D0043B9B1AF5D01360C368013BC360FB
:10375000C3691A44836902619A4224BF436A0361C0
:10376000002383620123E5E700F090B84FF0804327
:10377000002258631A610222DA6070474FF08043DA
:103780000022DA60704700004FF0804358637047B2
:103790004FF08043586A70474B6843608B68836082
:1037A000CB68C3600B6943614B6903628B694362F9
:1037B0000B6803607047000008B5224B22481A6965
:1037C00040F2FF110A431A611A6922F4FF7222F0D3
:1037D00001021A611A691A6B0A431A631A6D0A43C5
:1037E0001A651A4A1B6D1146FFF7D6FF184802F1F9
:1037F0001C01FFF7D1FF174802F13801FFF7CCFF9A
:10380000154802F15401FFF7C7FF144802F1700197
:10381000FFF7C2FF124802F18C01FFF7BDFF11480C
:1038200002F1A801FFF7B8FF0F4802F1C401FFF74A
:10383000B3FF0E4802F1E001FFF7AEFFBDE808401C
:1038400000F0AAB80038024000000240403F0008E3
:103850000004024000080240000C02400010024038
:103860000014024000180240001C024000200240E8
:1038700008B500F007FAFEF771FCFFF79BF8BDE80A
:103880000840FEF773BE000070470000104B1A6C32
:1038900042F001021A641A6E42F001021A660D4AE1
:1038A0001B6E936843F0010393604FF080435322F3
:1038B0009A624FF0FF32DA6200229A615A63DA604C
:1038C0005A6001225A6108211A601C20FDF75CBD74
:1038D00000380240002004E04FF0804208B5136930
:1038E000D1680B40D9B2C9439B07116107D520238A
:1038F00083F31188FEF752FC002383F3118808BD7F
:1039000008B5FFF7E9FFBDE80840FFF799B80000E8
:103910001F4B1A696FEAC2526FEAD2521A611A69D2
:10392000C2F308021A614FF0FF301A695A695861F0
:1039300000215A6959615A691A6A62F080521A6202
:103940001A6A02F080521A621A6A5A6A58625A6AED
:1039500059625A6A1A6C42F080521A641A6E42F026
:1039600080521A661A6E0B4A106840F4807010601C
:10397000186F00F44070B0F5007F1EBF4FF4803028
:1039800018671967536823F40073536000F05AB93D
:103990000038024000700040334B4FF080521A64F0
:1039A000324A4FF4404111601A6842F001021A6035
:1039B0001A689207FCD59A6822F003029A602A4B93
:1039C00019469A6812F00C02FBD1186800F0F90051
:1039D00018609A601A6842F480321A600B689B0380
:1039E000FCD54B6F43F001034B671F4B5A6F900799
:1039F000FCD51F4A5A601A6842F080721A601B4A4E
:103A000053685904FCD5184B1A689201FCD5194A21
:103A10009A60194B1A68194B9A42194B21D1194ACD
:103A20001168194A91421CD140F205121A60144AD9
:103A3000136803F00F03052BFAD10B4B9A6842F081
:103A400002029A609A6802F00C02082AFAD15A6CB3
:103A500042F480425A645A6E42F480425A665B6E67
:103A6000704740F20572E1E7003802400070004004
:103A70000854400700948838002004E011640020B6
:103A8000003C024000ED00E041C20F41084A08B589
:103A9000536911680B4003F00103536123B1054AD8
:103AA00013680BB150689847BDE80840FEF7C8BFDF
:103AB000003C0140D4230020084A08B5536911682E
:103AC0000B4003F00203536123B1054A93680BB125
:103AD000D0689847BDE80840FEF7B2BF003C0140FF
:103AE000D4230020084A08B5536911680B4003F03D
:103AF0000403536123B1054A13690BB15069984718
:103B0000BDE80840FEF79CBF003C0140D4230020E4
:103B1000084A08B5536911680B4003F00803536164
:103B200023B1054A93690BB1D0699847BDE80840B5
:103B3000FEF786BF003C0140D4230020084A08B5A8
:103B4000536911680B4003F01003536123B1054A18
:103B5000136A0BB1506A9847BDE80840FEF770BF82
:103B6000003C0140D4230020174B10B55C691A6853
:103B7000144004F478725A61A30604D5134A936A78
:103B80000BB1D06A9847600604D5104A136B0BB18D
:103B9000506B9847210604D50C4A936B0BB1D06B40
:103BA0009847E20504D5094A136C0BB1506C98474D
:103BB000A30504D5054A936C0BB1D06C9847BDE8BA
:103BC0001040FEF73DBF00BF003C0140D423002061
:103BD0001A4B10B55C691A68144004F47C425A61AF
:103BE000620504D5164A136D0BB1506D9847230535
:103BF00004D5134A936D0BB1D06D9847E00404D5FA
:103C00000F4A136E0BB1506E9847A10404D50C4AAD
:103C1000936E0BB1D06E9847620404D5084A136FB7
:103C20000BB1506F9847230404D5054A936F0BB12D
:103C3000D06F9847BDE81040FEF702BF003C01403E
:103C4000D4230020062108B50846FDF79DFB062178
:103C50000720FDF799FB06210820FDF795FB0621BB
:103C60000920FDF791FB06210A20FDF78DFB0621B7
:103C70001720FDF789FB06212820BDE80840FDF745
:103C800083BB000008B5FFF743FEFDF793F9FDF78E
:103C900021FDFDF70DFFFDF7E1FDFFF7F5FDBDE8A7
:103CA0000840FFF761BD0000034611F8012B03F83F
:103CB000012B002AF9D170471210121312110000C3
:103CC00053544D3332463F3F3F0000000000000098
:103CD000C03C00083F00000013040000143D000831
:103CE0003F000000190400001E3D00083F000000D6
:103CF00021040000283D00083F0000001832002089
:103D000054240020BC260020242900208C2B0020D5
:103D1000F42D002053544D33324634307800535440
:103D20004D3332463432780053544D3332463434B6
:103D30003658580000960000000000000000000007
:103D40000000000000000000000000009D160008B8
:103D500089160008C5160008B1160008BD1600082F
:103D6000A91600089516000881160008D11600084B
:103D700000000000D5170008C1170008FD17000853
:103D8000E9170008F5170008E1170008CD1700082B
:103D9000B9170008591800080000000001000000D1
:103DA000000000006D61696E00000000C43D000865
:103DB000A030002018320020010000005921000826
:103DC0000000000069646C65000000000200000053
:103DD00000000000011A0008691A000840004000B5
:103DE000B0360020C03600200200000000000000B5
:103DF0000300000000000000AD1A000800000000F1
:103E000010000000D036002000000000010000007B
:103E10000000000074390020010102004172647545
:103E200050696C6F740025424F415244252D424C1D
:103E3000002553455249414C250000000D2500083E
:103E4000752400086D190008F124000843000000E3
:103E5000543E000809024300020100C03209040078
:103E600000010202010005240010010524010001E7
